:100000000C9438050C947F050C947F050C947F05A7
:100010000C947F050C947F050C947F050C947F0550
:100020000C947F050C947F050C947F050C944E0F67
:100030000C94FD0F0C94F01D0C947F050C947F051F
:100040000C947F050C947F050C947F050C94641E22
:100050000C947F050C947F050C947F050C947F0510
:100060000C947F050C947F050C947F050C947F0500
:100070000C947F056A108C107A118C107A11D110B3
:10008000F4107A1149115C11D014D014FD14FD1430
:10009000581594158C178C17AC158C17A716A71626
:1000A00062178C178C177817041607090B0A1D1B8B
:1000B00006196405141A08151C171E1F2021232277
:1000C0002E26242D25273012182F0C13280F0D341F
:1000D0000E333136381110372B2C352A5829787BBE
:1000E00079397A504F5152726C63685680668053EA
:1000F000020103555880576D6E5462595A5B5C5D1E
:100100005E5F6F60617475663E3F403C414277447C
:1001100076466B47804365458048494A4B4C3D4D88
:100120003B4E3A7D7E7C7F730A0025303862003A70
:1001300020002530325800722F63203031323334A2
:100140003536370A006164625F686F73745F6B6293
:10015000645F726563763A204552524F5228256497
:10016000290A000A0025303458006164625F686F14
:1001700073745F6B62645F726563763A2000455208
:10018000524F523A206D65646961206B6579300A7F
:10019000004552524F523A206D65646961206B658B
:1001A00079310A005D0A0025640020002564007C86
:1001B000002530325800200025303258006164623A
:1001C0005F6D6F757365207261773A205B000A007E
:1001D0002530313662006164625F686F73745F6DF1
:1001E0006F7573655F726563763A2000646562754A
:1001F0006720656E61626C65642E0A005363616EF0
:100200003A20616464723A25642C20726567333A3F
:10021000253034580A00416674657220696E69742D
:100220003A0A00466F756E643A206D656469612014
:100230006B6579730A005363616E3A20616464727E
:100240003A25642C20726567333A253034580A0009
:100250004265666F726520696E69743A0A005B7365
:100260005D004B6579626F617264207374617274B2
:100270002E0A0055534220636F6E6669677572657A
:10028000642E0A005B575D005B535D005B525D00AE
:100290002E0341004400420020006B0065007900FD
:1002A00062006F00610072006400200063006F0054
:1002B0006E00760065007200740065007200000038
:1002C0000E0374002E006D002E006B002E00000047
:1002D0000403090409027400040100A032090400A7
:1002E0000001030101000921110100012240000762
:1002F00005810308000A0904010001030102000945
:100300002111010001224D000705820308000A099E
:10031000040200010300000009211101000122363E
:10032000000705830308000A090403000203000014
:100330000009211101000122220007058403200089
:10034000010705040320000112011001000000084C
:10035000EDFEDB0A0101010200010631FF0974A173
:10036000010975150026FF009520750881020976A0
:10037000150026FF00952075089102C0050109802F
:10038000A101850216810026B7001A81002AB70054
:10039000751095018100C0050C0901A101850316A6
:1003A0000100269C021A01002A9C02751095018109
:1003B00000C005010902A1010901A10005091901F7
:1003C0002905150025019505750181029501750323
:1003D00081010501093009311581257F95027508D4
:1003E000810609381581257F950175088106050C60
:1003F0000A38021581257F950175088106C0C00560
:10040000010906A101050719E029E7150025019555
:1004100008750181029501750881010508190129F6
:10042000059505750191029501750391010507195F
:100430000029FF150026FF00950675088100C00AF7
:10044000002530325820006B6579626F6172645FFD
:100450007265706F72743A20004C45443A20253022
:1004600032580A00290A002575002F002575005D05
:100470002800256400200025640020002564002059
:10048000002564007C0025303258006D6F7573655F
:100490006B6579205B62746E7C78207920762068A9
:1004A0005D287265702F61636C293A205B006D6B6B
:1004B0005F776865656C5F74696D655F746F5F6DAC
:1004C0006178203D2025640A006D6B5F7768656563
:1004D0006C5F6D61785F7370656564203D20256495
:1004E0000A006D6B5F74696D655F746F5F6D617835
:1004F000203D2025640A006D6B5F6D61785F73702D
:10050000656564203D2025640A006D6B5F696E742B
:10051000657276616C203D2025640A006D6B5F6416
:10052000656C6179203D2025640A006D6B5F7768FA
:1005300065656C5F74696D655F746F5F6D61782070
:100540003D2025640A006D6B5F776865656C5F6DA3
:1005500061785F7370656564203D2025640A006DD5
:100560006B5F74696D655F746F5F6D6178203D20AE
:1005700025640A006D6B5F6D61785F7370656564FB
:10058000203D2025640A006D6B5F696E746572768C
:10059000616C203D2025640A006D6B5F64656C61B1
:1005A00079203D2025640A000A00257500363A208E
:1005B000776865656C5F74696D655F746F5F6D61A9
:1005C000783A20000A00257500353A20776865657D
:1005D0006C5F6D61785F73706565643A20000A0036
:1005E000257500343A2074696D655F746F5F6D61C5
:1005F000783A20000A00257500333A206D61785F53
:1006000073706565643A20000A00257500323A204F
:10061000696E74657276616C286D73293A20000AE0
:1006200000257500313A2064656C6179282A3130E3
:100630006D73293A20000A092D2056616C75657387
:10064000202D0A004D3E004D25643E20003F0073E2
:1006500065742064656661756C740A00433E200011
:1006600077686572652064656C74613A20637572A1
:10067000736F723D25642C20776865656C3D256439
:100680000A53656520687474703A2F2F656E2E7753
:10069000696B6970656469612E6F72672F77696B2A
:1006A000692F4D6F7573655F6B6579730A000A0971
:1006B0002D204D6F7573656B6579202D0A45534369
:1006C0002F713A09717569740A313A0964656C6170
:1006D00079282A31306D73290A323A09696E7465B6
:1006E0007276616C286D73290A333A096D61785FFF
:1006F00073706565640A343A0974696D655F746F77
:100700005F6D61780A353A09776865656C5F6D6180
:10071000785F73706565640A363A09776865656C59
:100720005F74696D655F746F5F6D61780A0A703A16
:10073000097072696E742076616C7565730A643A2B
:10074000097365742064656661756C74730A7570ED
:100750003A092B310A646F776E3A092D310A7067B6
:1007600075703A092B31300A7067646F776E3A09F9
:100770002D31300A0A7370656564203D2064656C14
:100780007461202A206D61785F7370656564202A2A
:100790002028726570656174202F2074696D655F13
:1007A000746F5F6D6178290A003F004D3E20004361
:1007B0003E20004C25640A000A092D20436F6E7309
:1007C0006F6C65202D0A4553432F713A0971756985
:1007D000740A6D3A096D6F7573656B65790A000A65
:1007E000092D204D61676963202D0A643A0964650B
:1007F0006275670A783A096465627567206D61748D
:100800007269780A6B3A096465627567206B65796D
:10081000626F6172640A6D3A096465627567206D82
:100820006F7573650A763A0976657273696F6E0A39
:10083000733A097374617475730A633A09636F6E6E
:10084000736F6C65206D6F64650A302D343A096CE6
:1008500061796572302D34284631302D4634290AAD
:10086000506175733A09626F6F746C6F6164657281
:100870000A003F0074696D65725F726561643332AE
:1008800028293A202530346C580A006B6579626F4C
:100890006172645F69646C653A2025580A006B6573
:1008A00079626F6172645F70726F746F636F6C3ABC
:1008B0002025580A00686F73745F6B6579626F61F9
:1008C00072645F6C65647328293A2025580A000A0F
:1008D000092D20537461747573202D0A004743431A
:1008E0003A20342E392E32204156522D4C49424363
:1008F0003A20312E382E3073766E204156525F41A9
:100900005243483A2061767233350A004F505449B9
:100910004F4E533A204C554641204D4F5553454B71
:1009200045592045585452414B455920434F4E5349
:100930004F4C4520434F4D4D414E44204B45594D62
:1009400041505F53454354494F4E20343039360AA5
:10095000004255494C443A203330613166643120BD
:100960002831303A33303A333420536570203239ED
:100970002032303136290A005649443A2030784630
:1009800045454428742E6D2E6B2E29205049443A3B
:100990002030783041444228414442206B657962DE
:1009A0006F61726420636F6E766572746572292060
:1009B0005645523A203078303130310A00444553A0
:1009C000433A20636F6E7665727420414442206B17
:1009D0006579626F61726420746F205553420A001A
:1009E0000A092D2056657273696F6E202D0A000A60
:1009F0006D6F7573653A206F66660A000A6D6F75D4
:100A000073653A206F6E0A000A6B6579626F6172D6
:100A1000643A206F66660A000A6B6579626F6172DC
:100A2000643A206F6E0A000A6D61747269783A2028
:100A30006F66660A000A6D61747269783A206F6E9B
:100A40000A000A64656275673A206F6E0A000A64DC
:100A5000656275673A206F66660A000A0A626F6F00
:100A6000746C6F616465722E2E2E2000433E200050
:100A700011241FBECFEFD4E0DEBFCDBF04B603FE0E
:100A800027C08091DC019091DD01A091DE01B09141
:100A9000DF018730904BA740B04BD1F41092DC01BE
:100AA0001092DD011092DE011092DF0114BE84B7B6
:100AB000877F84BF0FB6F894A89580916000886105
:100AC00080936000109260000FBEE0E0F8E30995AB
:100AD00011E0A0E0B1E0E8EEFDE402C005900D9267
:100AE000A433B107D9F721E0A4E3B1E001C01D921E
:100AF000AC3DB207E1F70E949B0C0C94F2260C94DB
:100B00000000FF93EF93E0913401F09135013097AD
:100B100009F00995EF91FF910895FC0185918030CE
:100B200011F0EFDFFBCF0895FF27E0E230E247FF4F
:100B30000CC0419597FF09C0EDE2609570958095D6
:100B40009095611D711D811D911D27FF02C021958A
:100B500030E350E2AA27660F771F881F991FAA1F4C
:100B6000A41710F0A41B63955A95A9F7AA3008F0B2
:100B7000A95FA05DAF93F39561157105810591059E
:100B800041F7ED3211F4EF93F395F21718F43F9318
:100B9000F395FBCF8F91B5DFFA95E1F70895E991D1
:100BA000F9918591803021F0853219F0AADFF9CFD3
:100BB000089520E0E89455915532C1F3503311F473
:100BC000689455915A3348F4505390F3220F022EF3
:100BD000220F220F200D250FF4CF0EF421958991BD
:100BE0009991533619F3533729F1533559F1BC0113
:100BF00088279927E8945C3621F489919991689423
:100C00005591543639F446EF7EF077FF0DC08FEFE3
:100C10009FEF0AC055374AE039F0583540E121F0DE
:100C2000523642E009F00895FF93EF937DDFEF9194
:100C3000FF91B7CFFF93EF93FC0181918030B9F31F
:100C400060DFFBCFFF93EF9368DFF1CFDF93CF93AC
:100C5000CDB7DEB72596A3DFCF91DF910895282F7A
:100C60002770E82FE695E695E695EF70F0E0E95CF1
:100C7000FE4F87FF0AC081E090E001C0880F2A95EF
:100C8000EAF780959081892308C081E090E001C057
:100C9000880F2A95EAF79081892B808381E08093E1
:100CA0004C0108950F931F93CF93DF93569A5E9A4A
:100CB0000E9499092FEF87EA91E6215080409040E9
:100CC000E1F700C0000080E592E09F938F930E94BF
:100CD00026060F900F90C1E0D0E006E312E063E03B
:100CE0008C2F0E949D09009771F09F938F93DF9343
:100CF000CF931F930F930E9426060F900F900F9093
:100D00000F900F900F909FEF29EF80E091502040BF
:100D10008040E1F700C000002196C031D105F9F60E
:100D200063E082E00E949D098131910511F170F428
:100D300087309105F1F020F404970297F0F419C080
:100D400089309105B1F00D97C1F413C08D31910533
:100D500081F030F48431910561F0499771F409C054
:100D6000843C910531F0873C910519F0813C910557
:100D700021F481E080934D0102C010924D0163E0A7
:100D800087E00E949D0991E0823009F090E0909305
:100D90004E01992341F083E292E09F938F930E944A
:100DA00026060F900F9023E042E063E082E00E946D
:100DB0001D0A86E192E09F938F930E9426060F9072
:100DC0000F90C1E0D0E00CEF11E063E08C2F0E94A7
:100DD0009D09009771F09F938F93DF93CF931F939B
:100DE0000F930E9426060F900F900F900F900F9078
:100DF0000F908FEF99EF20E0815090402040E1F775
:100E000000C000002196C031D105F9F6E7E3F1E01A
:100E100080E18E0F11928E13FDCF0E9497110E94D8
:100E200040098091BE0181608093BE018CEE91E00B
:100E30000E948D05569A5E98DF91CF911F910F9178
:100E40000895CF93DF938FE79BEB0197F1F700C0F5
:100E500000000E94190AEC01009711F481E0BDC066
:100E600097FD05C080914701816080934701D7FFBE
:100E700005C0809147018E7F80934701ED2FFF27AA
:100E8000EF73FF27CE018F739927C6FF02C08054EE
:100E90009109D6FF02C0E054F109A09136010A2E53
:100EA000000CBB0BBD010E94A72681382FEF9207D3
:100EB00014F481E89FEF22273327281B390B2138B0
:100EC0008FEF380714F421E83FEF21952093480174
:100ED000CF01BD010E94A72681382FEF920714F49D
:100EE00081E89FEF91958195910981382FEF9207C5
:100EF00014F481E89FEF8195809349018091BE01B0
:100F000083FF60C086ED91E00E948D05DF93CF9353
:100F100080ED91E09F938F930E9426068EEC91E0E6
:100F20000E948D058DEB91E00E948D058091360128
:100F3000282F082E000C330B3F938F9388EB91E002
:100F40009F938F930E94260686EB91E00E948D0569
:100F5000809147011F928F9381EB91E09F938F9334
:100F60000E9426068FEA91E00E948D05809148013B
:100F7000282F082E000C330B3F938F938CEA91E0BF
:100F80009F938F930E9426068AEA91E00E948D0526
:100F900080914901282F082E000C330B3F938F932B
:100FA00087EA91E09F938F930E94260684EA91E05E
:100FB0000E948D058DB79EB744960FB6F8949EBFDC
:100FC0000FBE8DBF87E491E00E94EC118091360145
:100FD00091E088300CF090E0890F80933601DF912A
:100FE000CF9108951F93CF93DF9310924C01C0913E
:100FF0000001D09101018FEF9FEF90930101809349
:101000000001CF3F8FEFD80709F06AC08FE79BEB55
:101010000197F1F700C0000082E00E94160AEC017F
:10102000892B09F05DC080914E01882309F458C0D6
:1010300087E00E94160A009709F452C09C012F779E
:10104000332722303105A1F048F42115310569F02C
:101050002130310599F480788A641AC02330310533
:1010600051F02F373105A1F009C08078826410C09B
:10107000807889640DC0807888640AC081E991E035
:101080009F938F930E9426060F900F9081E18FC04F
:10109000292F33272F7733272130310579F050F06E
:1010A0002230310579F02330310581F4EC01D0781C
:1010B000D86416C0EC01D078D26412C0EC01D078AC
:1010C000DA640EC0EC01D078D9640AC08EE791E0F2
:1010D0009F938F930E9426060F900F9080E167C028
:1010E0008091BE0181FF18C0209709F45DC08AE697
:1010F00091E00E948D05DF93CF9385E691E09F9369
:101100008F930E94260683E691E00E948D050F9042
:101110000F900F900F9003C0209709F445C0CF3770
:101120009FE7D90711F48FE705C0CF3F8FEFD807AE
:1011300021F48FEF0E942F0639C02D2F3327822FE5
:101140001C2F2F3F310581F4DF93CF9385E491E08D
:101150009F938F930E9426060E9452060F900F9035
:101160000F900F908C2F23C090914D01992381F007
:10117000A9014F7755274233510521F42078822F5A
:101180008A6006C04A30510519F42078822F8263A4
:101190000E942F061F3F51F0DC2FCC27CF6FD0933A
:1011A0000101C093000102C080E001C081E0DF9135
:1011B000CF911F910895E82FF0E0E95CFE4F208168
:1011C000822F90E021E030E002C0220F331F6A95A9
:1011D000E2F72823392381E0232B09F480E00895E6
:1011E000E82FF0E0E95CFE4F80810895CF92DF9216
:1011F000EF92FF920F931F93CF93DF938091BE01E5
:1012000081FF35C087E391E00E948D0587E3E82EDA
:1012100081E0F82EC0E0D0E092E3C92E91E0D92E13
:101220000AE211E0DF93CF93DF92CF920E9426066D
:101230008FE291E00E948D05F70181917F010E946C
:10124000891D1F928F931F930F930E94260688E299
:1012500091E00E948D0521968DB79EB708960FB636
:10126000F8949EBF0FBE8DBFC031D105D9F6DF9176
:10127000CF911F910F91FF90EF90DF90CF90089545
:10128000682F609582E00C94560A509A83E091E0B2
:101290000197F1F700C0000050989AEB9A95F1F78A
:1012A00000C00895509A8AEB8A95F1F700C05098D3
:1012B00083E091E00197F1F700C000000895EF92FC
:1012C000FF920F931F93CF93DF93C0E0D0E090E89D
:1012D000E92EF12C082F10E0C7010C2E02C09595C5
:1012E00087950A94E2F780239123892B19F00E94B5
:1012F000520902C00E9445092196C830D10561F704
:10130000DF91CF911F910F91FF90EF900895489B2F
:1013100006C023E02A95F1F700000197C1F7089570
:10132000489906C023E02A95F1F700000197C1F71C
:1013300008955898509808950895CF92DF92EF92AB
:10134000FF920F931F93CF93DF9300D0CDB7DEB7FB
:10135000F894509AE3EFFBE03197F1F700C00000FA
:101360006A8389830E9452096A816C6089818295AF
:10137000807F862B0E945F090E94450984EF91E0DF
:101380000E949009892B21F4789482EE9FEF43C04C
:1013900084EF91E00E948709009711F478943BC094
:1013A00011E1C12CD12C02E882E890E00E94900962
:1013B0007C01882351F199270E948709882329F10C
:1013C000CC0CDD1C902F9E19E81A9E1518F4689419
:1013D000C0F806C0113121F478948CEE9FEF1BC049
:1013E000115011F78FE591E00E949009892B21F4AB
:1013F00078948BEE9FEF0FC08BE590E00E948709F9
:10140000892BB1F77894C60106C07894812F90E0BB
:101410009195819591090F900F90DF91CF911F9138
:101420000F91FF90EF90DF90CF90089560E00C94C3
:101430009D0960E083E00C949D091F93CF93DF9397
:1014400000D01F92CDB7DEB7182FF894509A83EFD3
:101450009BE00197F1F700C000002B834A8369836A
:101460000E9452096981862F88601295107F812B16
:101470000E945F090E9445098FE193E00197F1F70F
:1014800000C000000E9452094A81842F0E945F0917
:101490002B81822F0E945F090E94450978940F904A
:1014A0000F900F90DF91CF911F910895262F2770F5
:1014B00040E062E00C941D0A80915A0108959FB7A4
:1014C000F894109251019FBF9091D301943009F08C
:1014D00057C09091E9009F703091EC00232F21704C
:1014E00030FD20E8922B24E02093E9002091EB00CE
:1014F00020FF43C02091EE0027FF3FC020914F0105
:10150000222321F02091E80025FF37C010924F01DF
:1015100026E03091E80035FD15C03091D30134301C
:1015200061F53091EB0035FD28C0215021F481E0B8
:1015300080934F0122C0EFE9FFE03197F1F700C03F
:101540000000E7CF8093F1008091E80085FD0AC09C
:101550008091E80080FFFCCF8091E8008E77809337
:10156000E80006C08FB7F89421E0209351018FBFA7
:101570009F709093E90080E008959F709093E90038
:101580008FEF0895CF93DF9300D01F92CDB7DEB7D2
:101590009C018091D301843019F593E099833B83BA
:1015A0002A839093E9008FEF9091E800815095FD98
:1015B00006C095ED9A95F1F700008111F5CF809165
:1015C000E80085FF0DC040E050E063E070E0CE0130
:1015D00001960E945C0D8091E8008E778093E80070
:1015E0000F900F900F90DF91CF910895CF93DF93DD
:1015F00000D01F92CDB7DEB72091D301243021F562
:1016000022E029839B838A8383E08093E9008FEF24
:101610009091E800815095FD06C095ED9A95F1F7FF
:1016200000008111F5CF8091E80085FF0DC040E0FA
:1016300050E063E070E0CE0101960E945C0D809165
:10164000E8008E778093E8000F900F900F90DF9165
:10165000CF9108952091D3012430F1F422E020931A
:10166000E9002FEF3091E800215035FD06C035ED3F
:101670003A95F1F700002111F5CF2091E80025FF00
:101680000BC040E050E065E070E00E945C0D80918E
:10169000E8008E778093E8000895CF93DF93209140
:1016A000D301243039F521E02093E9002FEF309168
:1016B000E800215035FD06C035ED3A95F1F7000000
:1016C0002111F5CF2091E80025FF14C0EC0140E086
:1016D00050E068E070E00E945C0D8091E8008E7739
:1016E0008093E80088E0FE01A2E5B1E001900D9250
:1016F0008A95E1F7DF91CF9108958CE892E00C9400
:101700008D05209150012F5F822F62E30E94B82641
:10171000992319F02093500108951092500180915F
:101720005101882371F18091D301843041F580917A
:10173000E9008F702091EC00922F917020FD90E8CD
:10174000892B94E09093E9009091EB0090FF14C0F6
:101750009091EE0097FF10C09091E80095FF03C0B4
:101760001092F100F9CF9091E80090FF05C09091A0
:10177000E8009E779093E8008F708093E9001092C4
:101780005101089542E061EC81E00E94650E42E063
:1017900061EC82E00E94650E42E061EC83E00E9411
:1017A000650E42E261EC84E00C94650E8091D501F7
:1017B000833009F453C030F4813071F0823009F481
:1017C0008CC008958A3009F478C08B3009F45EC06B
:1017D000893009F09AC020C08091D401813A09F083
:1017E00094C08091E800877F8093E8008091D801C1
:1017F0009091D901892B21F468E082E591E003C042
:1018000060E080E090E070E00E94A70D8091E80029
:101810008B778093E80008958091D401813209F09C
:1018200074C08091D8019091D901892B09F06DC0C5
:101830008091E800877F8093E8008091E80082FD36
:1018400005C08091D3018111F8CF5FC08091F10074
:1018500080935A018091E8008B7753C08091D40126
:10186000813A09F052C08091D8019091D901892B19
:1018700009F04BC08091E800877F8093E800809159
:10188000E80080FFFCCF80910C0136C08091D4012C
:101890008132D9F58091D8019091D901892BA9F590
:1018A0008091E800877F8093E8000E949A0E8091E3
:1018B000D60180930C010C94AD178091D401813234
:1018C00021F58091E800877F8093E8000E949A0EBE
:1018D0008091D70180935B0108958091D401813A72
:1018E000A1F48091E800877F8093E8008091E80070
:1018F00080FFFCCF80915B018093F1008091E80034
:101900008E778093E8000C949A0E089508950895B8
:10191000089588E892E00E948D050C94880C0E943E
:10192000AF1D8091D101882329F00E94DA1D811119
:101930000C94460D089584B7877F84BF0FB6F89442
:10194000A89580916000886180936000109260008B
:101950000FBE90E080E80FB6F894809361009093FA
:1019600061000FBE0E94860C0E9424120E94EB0EA2
:101970000E943E0F8091E20084608093E2008FE538
:101980009AE00E94841D78948091D3018430E1F71D
:1019900083E792E00E948D050E94261282E091E08A
:1019A0000E94921182E692E00E948D050E94870CAF
:1019B0008091D301853039F48EE592E00E948D0547
:1019C0000E948F0CF5CF0E942C12F2CF0C94EE1DCA
:1019D00084E892E00E948D050C94E60C292F3327B1
:1019E00023303105C9F064F42130310581F0223013
:1019F000310509F043C084E790E024ED32E042C0B5
:101A000021323105F1F02232310541F137C082E156
:101A100090E028E433E036C099278130910541F009
:101A20008230910541F0892B49F5E0EDF2E005C0E7
:101A3000E0ECF2E002C0E0E9F2E0849190E09F0186
:101A400021C06430D8F4E62FF0E0EE0FFF1FEF5D09
:101A5000FE4F2081318189E090E014C0643070F441
:101A600070E0FB01EE0FFF1FE75EFE4F208131812A
:101A7000FB01EB5EFE4F808190E004C080E090E0CF
:101A800020E030E0FA0131832083089584E089BDAD
:101A900086E089BD09B400FEFDCF8091D8008F7D1E
:101AA0008093D8008091E00082608093E000809174
:101AB000E00081FDFCCF0895CF92DF92EF92FF927C
:101AC0000F931F93CF93DF93EC018B016A010E9468
:101AD000B90E811133C0C114D10439F0F6018081EF
:101AE0009181081B190BC80FD91FE12CF12C01158E
:101AF000110519F18091E80085FD16C08091E8007C
:101B00008E778093E800C114D10449F0F6018081FA
:101B10009181E80EF91EF182E08285E00FC00E94FB
:101B2000B90E882321F30AC089918093F1000150F6
:101B30001109FFEFEF1AFF0ADACF80E0DF91CF91B2
:101B40001F910F91FF90EF90DF90CF90089520911B
:101B5000DA013091DB012617370748F0611571056E
:101B600039F42091E8002E772093E80001C0B901F4
:101B700040E06115710591F12091D301222309F410
:101B800040C0253009F43FC02091E80023FD3DC04E
:101B90002091E80022FD2FC02091E80020FFE9CF2E
:101BA0002091F20030E0FC01CF016115710559F080
:101BB0002830310540F481918093F1006150710922
:101BC0002F5F3F4FF1CF41E02830310509F040E071
:101BD0002091E8002E772093E800CBCF4111CCCFA5
:101BE0000AC08091D301882361F0853061F0809133
:101BF000E80083FD0AC08091E80082FFF2CF80E018
:101C0000089582E0089583E0089581E00895209189
:101C1000DA013091DB012617370748F061157105AD
:101C200039F42091E8002E772093E80001C0B90133
:101C3000FC0120E06115710579F18091D3018823C1
:101C400009F43DC0853009F43CC08091E80083FD73
:101C50003AC08091E80082FD2CC08091E80080FFAE
:101C6000E9CF8091F20090E06115710559F088305C
:101C7000910540F424912093F1003196615071094F
:101C80000196F2CF21E0089709F020E08091E8006A
:101C90008E778093E800CECF2111CFCF0AC08091FC
:101CA000D301882361F0853061F08091E80083FDE5
:101CB0000AC08091E80082FFF2CF80E0089582E0C0
:101CC000089583E0089581E00895982F953058F5A0
:101CD0009093E900981739F07091EC002091ED0095
:101CE0005091F00003C0242F762F50E021FF19C03F
:101CF0003091EB003E7F3093EB003091ED003D7F63
:101D00003093ED003091EB0031603093EB00709335
:101D1000EC002093ED005093F0002091EE0027FF9F
:101D200007C09F5FD3CF8F708093E90081E0089553
:101D300080E008958091D40187FF11C08091E80070
:101D400082FD05C08091D3018111F8CF11C080912F
:101D5000E8008B770BC08091D301882349F08091F4
:101D6000E80080FFF8CF8091E8008E778093E8004C
:101D700008952091E4003091E50095E64091EC0053
:101D8000842F817040FF22C08091E80080FD1CC03C
:101D90008091D301882391F0853091F08091EB0000
:101DA00085FD10C04091E4005091E50042175307B3
:101DB00029F39A01915011F784E0089582E0089583
:101DC00083E0089581E0089580E008954091E8005F
:101DD00042FFDECF08950E94480F0E944B0FE0EEB5
:101DE000F0E0808181608083E8EDF0E080818F7792
:101DF000808319BCE3E6F0E08081816080831092EB
:101E0000D20108950E94480F0E944B0F8091D80084
:101E10008F778093D8008091D80080688093D80015
:101E20008091D8008F7D8093D80084E089BD86E0C2
:101E300089BD09B400FEFDCF1092D3011092CF01ED
:101E40001092D1011092D00142E060E080E00E9447
:101E5000650E8091E1008E7F8093E1008091E20029
:101E600081608093E2008091E20088608093E200CC
:101E70008091E0008E7F8093E0000895E3E6F0E03B
:101E800080818E7F808381E08093D2010C94020F49
:101E90001092E20008951092E10008951F920F92AF
:101EA0000FB60F9211242F933F934F935F936F932D
:101EB0007F938F939F93AF93BF93EF93FF93809103
:101EC000E10082FF0BC08091E20082FF07C0809199
:101ED000E1008B7F8093E1000E94810B8091E10003
:101EE00080FF19C08091E20080FF15C08091E20060
:101EF0008E7F8093E2008091E20080618093E20017
:101F00008091D80080628093D80019BC85E08093CE
:101F1000D3010E94890C8091E10084FF30C0809140
:101F2000E20084FF2CC084E089BD86E089BD09B44D
:101F300000FEFDCF8091D8008F7D8093D8008091E6
:101F4000E1008F7E8093E1008091E2008F7E80939C
:101F5000E2008091E20081608093E2008091CF01F5
:101F6000882311F084E007C08091E30087FD02C060
:101F700081E001C083E08093D3010E94E80C80914E
:101F8000E10083FF29C08091E20083FF25C080919A
:101F9000E100877F8093E10082E08093D30110927B
:101FA000CF018091E1008E7F8093E1008091E2007B
:101FB0008E7F8093E2008091E20080618093E20056
:101FC00042E060E080E00E94650E8091F000886051
:101FD0008093F0000E947D0BFF91EF91BF91AF9134
:101FE0009F918F917F916F915F914F913F912F9131
:101FF0000F900FBE0F901F9018951F920F920FB663
:102000000F9211242F933F934F935F936F937F937E
:102010008F939F93AF93BF93CF93DF93EF93FF93F0
:10202000C091E900CF708091EC00D82FD17080FD75
:10203000D0E81092E9008091F000877F8093F00053
:1020400078940E9441101092E9008091F00088601D
:102050008093F000CD2BCF70C093E900FF91EF91FA
:10206000DF91CF91BF91AF919F918F917F916F91B0
:102070005F914F913F912F910F900FBE0F901F9046
:1020800018951F93CF93DF93CDB7DEB7AA970FB6FE
:10209000F894DEBF0FBECDBFE4EDF1E088E08E0F17
:1020A0009091F10091938E13FBCF0E94D60B8091FB
:1020B000E80083FF1FC18091D4019091D501492F81
:1020C00050E04A30510508F015C1FA01E65CFF4FB7
:1020D0000C94D826803881F0823809F00BC18091A9
:1020E000D8018F708093E9008091EB0085FB8827F1
:1020F00080F91092E90006C08091D0019091D10141
:10210000911182609091E800977F9093E80080930E
:10211000F1001092F100C8C0282F2D7F09F0EAC00D
:10212000882319F0823061F0E5C08091D6018130BA
:1021300009F0E0C0933009F080E08093D1012BC01A
:102140008091D601811127C08091D8018F7009F448
:10215000D1C08093E9002091EB0020FF1CC0933098
:1021600021F48091EB00806214C09091EB009061AB
:102170009093EB0021E030E0A90102C0440F551F0D
:102180008A95E2F74093EA001092EA008091EB0012
:1021900088608093EB001092E9008091E800877FCF
:1021A00086C08111A7C01091D6011F778091E300EE
:1021B0008078812B8093E3008091E800877F809373
:1021C000E8000E949A0E8091E80080FFFCCF809189
:1021D000E30080688093E300111102C082E001C037
:1021E00083E08093D30186C08058823008F082C09B
:1021F0008091D6019091D7018C3D53E0950779F5F8
:1022000083E08A838AE289834FB7F894DE011396CC
:1022100020E03EE051E2E32FF0E050935700E491DC
:1022200020FF03C0E295EF703F5FEF708E2F90E0CC
:10223000EA3010F0C79601C0C0968D939D932F5F32
:10224000243149F74FBF8091E800877F8093E800F1
:102250006AE270E0CE0101960E94A70D14C0AE01A3
:102260004F5F5F4F6091D8010E94EE0CBC01892B3B
:1022700009F440C09091E800977F9093E80089812D
:102280009A810E94070E8091E8008B778093E80086
:1022900031C0803879F58091E800877F8093E8002D
:1022A0008091CF018093F1008091E8008E77809338
:1022B000E8000E949A0E1EC081111CC09091D601A8
:1022C0009230C0F48091E800877F8093E80090937B
:1022D000CF010E949A0E8091CF01811106C080919A
:1022E000E30087FD02C081E001C084E08093D30158
:1022F0000E94C20B8091E80083FF0AC08091E80031
:10230000877F8093E8008091EB0080628093EB00F0
:10231000AA960FB6F894DEBF0FBECDBFDF91CF9166
:102320001F91089590936101809360010895E09159
:102330006001F0916101309721F00190F081E02D72
:10234000099480E00895EF92FF920F931F93CF932B
:10235000DF93E0916001F09161013097B1F18C0160
:102360000280F381E02D09958091BE0182FF2DC08E
:1023700080FF04C087E494E00E948D05E80118E026
:1023800081E4E82E84E0F82E8091BE0180FF0BC02E
:1023900088811F928F93FF92EF920E9426060F90E2
:1023A0000F900F900F90115021961111EDCF809149
:1023B000BE0180FF0AC08FE394E0DF91CF911F91AF
:1023C0000F91FF90EF900C948D05DF91CF911F91AD
:1023D0000F91FF90EF900895E0916001F0916101FD
:1023E000309721F00480F581E02D09940895209123
:1023F0005E0130915F018217930771F090935F0146
:1024000080935E01E0916001F0916101309721F0CD
:102410000680F781E02D0994089520915C013091A8
:102420005D018217930771F090935D0180935C01C9
:10243000E0916001F0916101309721F00084F18515
:10244000E02D0994089508950C9423120E94191EFA
:102450000E9452060C949C09CF92DF92EF92FF9259
:102460000F931F93CF93DF9300D000D000D0CDB750
:10247000DEB70E94F20783E6C82E81E0D82E00E086
:1024800010E0E02E802F0E94F008F60141916F01CC
:10249000F42EF826B1F40F5F1F4F0031110589F7B4
:1024A0008FEF89838A831B820E94221E8160782F8E
:1024B0009D838C8349815A816B818D810E94ED12AD
:1024C00047C09091BE0191FF04C08E830E94F60820
:1024D0008E8120E030E04F2D50E0922FBA01022E85
:1024E00002C0759567950A94E2F760FF2BC02983B7
:1024F000EA8221E030E0690102C0CC0CDD1C9A9533
:10250000E2F790E08C219D21892B09F420E02B83B8
:102510000E94221E8160782F9D838C8349815A817D
:102520006B818D810E94ED1249815A816B817C8182
:102530008D810E949C1DF801ED59FE4F8081C826B7
:10254000C08206C02F5F3F4F2830310531F6A3CF40
:102550000E949B1D0E94EF200E94210710916201A2
:102560000E949711181741F10E9497118093620100
:102570009091BE0192FF0EC090FF0CC01F928F93EE
:1025800089E594E09F938F930E9426060F900F9009
:102590000F900F908091620126960FB6F894DEBFDF
:1025A0000FBECDBFDF91CF911F910F91FF90EF90A4
:1025B000DF90CF900C94AD1D26960FB6F894DEBF39
:1025C0000FBECDBFDF91CF911F910F91FF90EF9084
:1025D000DF90CF9008950C944009CF93DF93CDB74F
:1025E000DEB72B970FB6F894DEBF0FBECDBF942F8A
:1025F0004F83252F588769877A878B874A855B8524
:10260000452B21F02F3F09F59F3FF9F4DE0111968C
:1026100086E0FD0111928A95E9F785E0FE01379683
:1026200001900D928A95E1F749815A816B817C81F5
:102630008D819E810E94561A2B960FB6F894DEBFAC
:102640000FBECDBFDF91CF9108954F815885698529
:102650007A858B850E949C1DD9CFCF93882309F45E
:10266000E8C0C82F8238A1F40E94971181FDE1C013
:1026700089E30E94E51C0E945E1D2FEF81EE94E02D
:10268000215080409040E1F700C0000089E315C070
:102690008338C1F40E94971180FDCBC083E50E946E
:1026A000E51C0E945E1D2FEF81EE94E021508040DA
:1026B0009040E1F700C0000083E50E94021DCF9129
:1026C0000C945E1D8438A1F40E94971182FDB1C064
:1026D00087E40E94E51C0E945E1D2FEF81EE94E0CE
:1026E000215080409040E1F700C0000087E4E5CF32
:1026F0008CEF8C0F813A48F48C2F0E941B2481119F
:1027000098C08C2F0E94E51CDACF80E28C0F8830B5
:1027100048F4C77081E001C0880FCA95EAF70E94AB
:10272000241DCDCF8BE58C0F833078F4C53A29F08A
:10273000C63A31F083E890E005C081E890E002C03D
:1027400082E890E0CF910C94F71188E58C0F8531E9
:1027500008F06FC0C83A61F1C93A69F1CA3A71F13B
:10276000CB3A79F1CC3A81F1CD3A89F1CE3A91F177
:10277000CF3A99F1C13BA1F1C03BA9F1C23BB1F104
:10278000C33BB9F1C43BC1F1C53BC9F1C63BD1F173
:10279000C73BD9F1C83BE1F1C93BE9F1CA3BF1F1D3
:1027A000CB3BF9F1CC3B09F43FC080E090E03EC068
:1027B00082EE90E03BC089EE90E038C08AEE90E077
:1027C00035C085EB90E032C086EB90E02FC083EB04
:1027D00090E02CC084EB90E029C087EB90E026C00D
:1027E0008CEC90E023C08DEC90E020C083E891E079
:1027F0001DC08AE891E01AC082E991E017C084E91F
:1028000091E014C081E292E011C083E292E00EC038
:1028100084E292E00BC085E292E008C086E292E09A
:1028200005C087E292E002C08AE292E0CF910C9468
:102830000D12CF910895882309F466C08238A1F45F
:102840000E94971181FF60C089E30E94E51C0E94ED
:102850005E1D2FEF81EE94E0215080409040E1F723
:1028600000C0000089E315C08338B9F40E949711B5
:1028700080FF4AC083E50E94E51C0E945E1D2FEF89
:1028800081EE94E0215080409040E1F700C00000CC
:1028900083E50E94021D0C945E1D8438A1F40E9401
:1028A000971182FF31C087E40E94E51C0E945E1DE3
:1028B0002FEF81EE94E0215080409040E1F700C07E
:1028C000000087E4E6CF9CEF980F913A10F390E276
:1028D000980F983050F4877091E001C0990F8A9555
:1028E000EAF7892F0E942A1DD6CF9BE5980F9330D7
:1028F00020F480E090E00C94F711885A853120F4A0
:1029000080E090E00C940D120895882321F00E943D
:10291000241D0C945E1D0895882321F00E942A1D19
:102920000C945E1D0895CF92DF92EF92FF920F9369
:102930001F93CF93DF9300D000D000D0CDB7DEB788
:1029400025E0FC01DE01119601900D922A95E1F738
:10295000FC0140813181F280258122952F706381B5
:102960007481672B09F4D8C23F3F19F44F3F09F433
:10297000D3C26C0149833A8389819A812E830E9454
:10298000A41C182F092F0E94A31C0E94B31BE02F28
:10299000E295EF70F0E0EC5BFF4F2E810C94D826AF
:1029A000802F807F902F9F70092F882311F0029530
:1029B000007FFF2049F0002309F45FC2802F0E94AE
:1029C000371D0E945E1D59C2812F0E941B140023D7
:1029D00009F4A2C2802F0E943D1D26960FB6F894DE
:1029E000DEBF0FBECDBFDF91CF911F910F91FF9042
:1029F000EF90DF90CF900C945E1D802F807F902F02
:102A00009F70092F803211F00295007F112319F079
:102A1000113001F129C0FF20A9F0802F222349F1B4
:102A2000213039F526960FB6F894DEBF0FBECDBF24
:102A3000DF91CF911F910F91FF90EF90DF90CF909A
:102A40000C94471D222319F0213009F465C20E941D
:102A50004A1D2CC0FF20E9F0263008F05DC20E941C
:102A6000211D802329F022C0FF20F1F0211115C083
:102A7000802F26960FB6F894DEBF0FBECDBFDF9134
:102A8000CF911F910F91FF90EF90DF90CF900C941A
:102A90008514253008F040C209C0F601858180FF09
:102AA000ECC18F708583E4CF2111FBC1802F69C1F8
:102AB000202F26952695237030E02115310521F031
:102AC00021303105C9F028C2FF2021F0812F902F3D
:102AD000937002C080E090E026960FB6F894DEBFB7
:102AE0000FBECDBFDF91CF911F910F91FF90EF905F
:102AF000DF90CF900C94F711FF2021F0812F902FC1
:102B0000937002C080E090E026960FB6F894DEBF86
:102B10000FBECDBFDF91CF911F910F91FF90EF902E
:102B2000DF90CF900C940D12812FFF2019F00E949E
:102B3000751F02C00E94DD1F26960FB6F894DEBFF7
:102B40000FBECDBFDF91CF911F910F91FF90EF90FE
:102B5000DF90CF900C946220802F837009F078C0B2
:102B6000F110DAC1812F829586958770880F880FC2
:102B7000912F9F70C92ED12CE12CF12C082E04C06E
:102B8000CC0CDD1CEE1CFF1C0A94D2F714FF12C003
:102B90004FE050E060E070E004C0440F551F661F36
:102BA000771F8A95D2F7CB01BA0160957095809511
:102BB000909503C060E070E0CB01202F269526950C
:102BC0002370422F50E042305105D1F0433051057F
:102BD00059F16C297D298E299F294130510541F1F8
:102BE00026960FB6F894DEBF0FBECDBFDF91CF9112
:102BF0001F910F91FF90EF90DF90CF900C94C81B26
:102C00006C297D298E299F2926960FB6F894DEBF60
:102C10000FBECDBFDF91CF911F910F91FF90EF902D
:102C2000DF90CF900C94DA1B0E94C81BC701B6013D
:102C300026960FB6F894DEBF0FBECDBFDF91CF91C1
:102C40001F910F91FF90EF90DF90CF900C94B61BE7
:102C5000FF2019F0802F817001C08695882309F428
:102C60005BC1812F829586958770880F880F912F81
:102C70009F70C92ED12CE12CF12C082E04C0CC0C55
:102C8000DD1CEE1CFF1C0A94D2F714FF12C04FE0AB
:102C900050E060E070E004C0440F551F661F771FCE
:102CA0008A95D2F7CB01BA01609570958095909581
:102CB00003C060E070E0CB01202F2695269523709D
:102CC000422F50E042305105D1F04330510559F1C7
:102CD0006C297D298E299F294130510541F1269685
:102CE0000FB6F894DEBF0FBECDBFDF91CF911F911D
:102CF0000F91FF90EF90DF90CF900C947F1C6C2988
:102D00007D298E299F2926960FB6F894DEBF0FBE27
:102D1000CDBFDF91CF911F910F91FF90EF90DF908A
:102D2000CF900C94911C0E947F1CC701B60126967F
:102D30000FB6F894DEBF0FBECDBFDF91CF911F91CC
:102D40000F91FF90EF90DF90CF900C946D1C103F8F
:102D500041F118F4103E48F48BC0123F09F450C002
:102D6000D8F1133F09F460C083C01F70802F8F71AA
:102D7000FF2021F00E94061C812F7BCE0E94271C81
:102D8000812F26960FB6F894DEBF0FBECDBFDF9120
:102D9000CF911F910F91FF90EF90DF90CF900C9407
:102DA0008C14FF20A9F0253008F0B6C0802F8F7159
:102DB00026960FB6F894DEBF0FBECDBFDF91CF9140
:102DC0001F910F91FF90EF90DF90CF900C944C1CCF
:102DD000263008F0A1C0EACFFF20A1F0802F8F712C
:102DE00026960FB6F894DEBF0FBECDBFDF91CF9110
:102DF0001F910F91FF90EF90DF90CF900C94061CE5
:102E0000FF2061F3802F8F7126960FB6F894DEBFF6
:102E10000FBECDBFDF91CF911F910F91FF90EF902B
:102E2000DF90CF900C94271CFF2091F0802F8F71A2
:102E300026960FB6F894DEBF0FBECDBFDF91CF91BF
:102E40001F910F91FF90EF90DF90CF900C94F11BAA
:102E500026960FB6F894DEBF0FBECDBFDF91CF919F
:102E60001F910F91FF90EF90DF90CF900C94EC1B8F
:102E7000FF20A1F0222309F4B1CF812F26960FB6AF
:102E8000F894DEBF0FBECDBFDF91CF911F910F91A0
:102E9000FF90EF90DF90CF900C942D13222309F434
:102EA000B1CF812F26960FB6F894DEBF0FBECDBFEF
:102EB000DF91CF911F910F91FF90EF90DF90CF9016
:102EC0000C941B14402F4F70612FC6010E94EB1E03
:102ED00026960FB6F894DEBF0FBECDBFDF91CF911F
:102EE0001F910F91FF90EF90DF90CF900C94FE1AFE
:102EF000402F4F70612FC60126960FB6F894DEBFA3
:102F00000FBECDBFDF91CF911F910F91FF90EF903A
:102F1000DF90CF900C94EE1E26960FB6F894DEBF8D
:102F20000FBECDBFDF91CF911F910F91FF90EF901A
:102F3000DF90CF9008950E94441D0E94131D0E94AF
:102F40005E1D0E9496210E94622080E090E00E9417
:102F5000F71180E090E00C940D120E94341D0C9447
:102F60009B170E94A41C292F22952F7030E02C3033
:102F700031054CF42A3031056CF4225031092230ED
:102F8000310588F407C02C30310549F02F30310568
:102F900031F009C0803E48F0803F29F406C093FB21
:102FA000882780F9089580E0089581E00895CF93FF
:102FB000DF9300D000D01F92CDB7DEB70F900F90F7
:102FC0000F900F900F90DF91CF910895CF93DF93E3
:102FD00000D000D000D0CDB7DEB726960FB6F8945B
:102FE000DEBF0FBECDBFDF91CF910895CF93DF93AA
:102FF000C091730180917401C817A1F0D0E0CE0197
:1030000066E070E00E94A726FC01EB58FE4F40816D
:10301000518162817381848195810E94E617219696
:10302000C770E8CFDF91CF9108954091A5015091ED
:10303000A6016091A7017091A8018091A9019091CA
:10304000AA010C94E617CF93DF938091AA01829591
:103050008F7009F05CC08091A701882309F457C0E4
:1030600020917301D09174014091A501C091A601F6
:10307000E091A801F091A9012D1709F448C030E0B2
:10308000309709F440C0CF3F11F44F3FE1F1C9013F
:1030900066E070E00E94A726DC01AB58BE4F119697
:1030A0008C911197C8132FC08C9148132CC0129685
:1030B0008C911297811127C013968D919C91149732
:1030C0008E179F0708F401978E1B9F0B883C910574
:1030D000D0F48091AA018F7080618093AA01C90108
:1030E00066E070E00E94A726FC01E658FE4F908142
:1030F0009F709061908385EA91E00E949314DF9124
:10310000CF910C94F6172F5F3F4F2770B5CFDF910B
:10311000CF910895BF92CF92DF92EF92FF920F93DB
:103120001F93CF93DF93CDB7DEB761970FB6F894B7
:10313000DEBF0FBECDBF8C0185E0F801DE011D961C
:1031400001900D928A95E1F7D8014C9111962C913E
:1031500011971296EC9012971396CD90DC901497DD
:103160005091A5016091A6018091A8019091A901BB
:10317000009709F46EC16F3F19F45F3F09F469C10C
:10318000B090A701BB2009F4C3C03091AA01C816B2
:10319000D90628F0F601E81BF90BCF0104C0809591
:1031A00090958C0D9D1DFF24F394883C910588F02B
:1031B000F12C307F09F0CBC07C2DD98AC88A522FE0
:1031C0006E2D89890E94D71785EA91E00E94931499
:1031D000B4C0832F807F09F049C0621314C0541318
:1031E00012C0E11010C03F7030613093AA010E94FC
:1031F000151885EA91E00E9493148091AA01D801E4
:1032000015968C9331C0CD2831F12F3F11F44F3FEB
:1032100011F1FE2CE1101FC0E09173013091740197
:10322000E31709F45CC0F0E0CF0166E070E00E94B3
:10323000A726DC01AB58BE4F11968C91119728132D
:1032400007C08C91481304C012968C91811103C061
:103250003196E770E5CFFE2CEE2009F416C180917F
:10326000AA0181608093AA01F12C0FC1621308C0EA
:10327000541306C0E11004C08091AA01D801C1C056
:103280004D872E878D859E850E94B1178823E1F199
:10329000EE20D1F12091AA01822F82958F7090E0CB
:1032A000029774F08091A5019091A60198878F8371
:1032B0001986DB86CA862C87CE0107960E94931456
:1032C00086E0F801A5EAB1E001900D928A95E1F758
:1032D0000E9423180E941518FF24F394D6C04D872E
:1032E0002E878D859E850E94A41C292F22952F70E4
:1032F00030E0223031050CF0BCC09F7009F0B6C040
:10330000805E883008F4C1C0C8010E949314E4CFE5
:10331000C816D90608F453C0F601E81BF90BCF0113
:10332000883C910508F450C0F12C7C2DD98AC88ABC
:10333000522F6E2D89890E94D717E5EAF1E086E0C9
:10334000DF011D928A95E9F70E9415189EC062134D
:1033500014C0541312C0E11010C08091AA01F801EA
:103360008583C8010E94931486E0E5EAF1E0DF015D
:103370001D928A95E9F7FB2C88C04D872E878D8595
:103380009E850E94B117882309F4BECFEE2009F470
:10339000BBCF2091AA01822F82958F7090E0029777
:1033A0000CF48ECF8091A5019091A6019A83898318
:1033B0001B82DD82CC822E83CE0101967FCF809549
:1033C00090958C0D9D1DACCFFE2CEE2009F49CCF6A
:1033D00062132EC054132CC02091AA0120FD1FC0DF
:1033E000822F82958F70D9F0D80115962C9315975E
:1033F0008F3049F08F5F982F9295907F822F8F703A
:10340000892B15968C93C8010E94931486E0F801CD
:10341000A5EAB1E001900D928A95E1F795CF86E09B
:10342000F801A5EAB1E001900D928A95E1F72DC06F
:103430004D872E878D859E850E94B117811140CFC3
:103440008091AA0181608093AA01C8010E9493140F
:103450001CC0EE2009F458CF4D872E878D859E85A0
:103460000E94B117882309F44FCF2ACF811148CF8A
:103470000CC0243031050CF047CF9F7009F440CFC9
:10348000F8019581907F09F03BCF8F2D61960FB6A3
:10349000F894DEBF0FBECDBFDF91CF911F910F918A
:1034A000FF90EF90DF90CF90BF900895CF93DF9380
:1034B000CDB7DEB72C970FB6F894DEBF0FBECDBFE9
:1034C0004F83588769877A878B879C87CE010796B9
:1034D0000E948A18882371F08F8198852A853B8500
:1034E000232B09F43FC09F3F09F068C08F3F09F0CC
:1034F00065C038C086E0FE013796DE011196019066
:103500000D928A95E1F76F817885EA85FB85309782
:1035100049F17F3F11F46F3F29F18091740190E0F0
:103520009C012F5F3F4F277033274091730150E07C
:103530002417350709F44BC069837A83FD83EC8334
:1035400066E070E00E94A726DC01AB58BE4F96E013
:10355000FE01319601900D929A95E1F72093740146
:103560000E94F61780917301909174018917E9F117
:1035700090E066E070E00E94A7268B589E4F0E9464
:103580008A18882391F18091730190E066E070E0E1
:103590000E94A726FC01EB58FE4F408151816281B9
:1035A0007381848195810E94E6178091730190E078
:1035B00001968770992780937301D4CF4F815885E6
:1035C00069857A858B859C850E94E617CBCF0E9402
:1035D000AD171092740110927301E5EAF1E086E0F4
:1035E000DF011D928A95E9F7BDCF2C960FB6F894AE
:1035F000DEBF0FBECDBFDF91CF910895DF92EF9276
:10360000FF920F931F93CF93DF93FC01892B09F453
:103610008AC0E12CF12CDD24D394EF012196849112
:10362000853709F461C058F4843708F04EC08430FF
:1036300008F06AC08130D1F0823071F174C08837EF
:1036400009F45DC050F4863709F455C0873709F096
:103650006AC08E2D0E94311D54C09CE7980F903790
:1036600008F061C08F770E941B1450C08F010E5F5D
:103670001F4FFE01849190E2980F983050F48770AC
:10368000FD2D01C0FF0F8A95EAF78F2F0E94371D8D
:1036900014C00E942D1313C08F010E5F1F4FFE0137
:1036A000C49180E28C0F883060F4C7708D2D01C00A
:1036B000880FCA95EAF70E943D1D0E945E1DE80131
:1036C00025C08C2F0E941B14FACF9F012E5F3F4F05
:1036D000FE01C491CC2369F08FE99FE00197F1F7D7
:1036E00000C00000C150F6CF9F012E5F3F4FFE018A
:1036F000F490E9010BC00E94211DE82E07C00E9432
:10370000341D0E945E1D02C00E942D138F2D882340
:1037100041F0EFE9FFE03197F1F700C00000815080
:10372000F6CFFE017ACFDF91CF911F910F91FF90DD
:10373000EF90DF9008956093AF017093B001809394
:10374000B1019093B2010E94AB1D0C949B17609342
:10375000AB017093AC018093AD019093AE010E94D8
:10376000AC1D0C949B1708950C949B1B0F931F93F7
:103770000091AF011091B0012091B1013091B201DF
:10378000602B712B822B932B1F910F910C949B1B01
:103790000F931F930091AF011091B0012091B101DF
:1037A0003091B20160237123822393231F910F91E3
:1037B0000C949B1B0F931F930091AF011091B001CC
:1037C0002091B1013091B2016027712782279327A0
:1037D0001F910F910C949B1B60E070E0CB010C9447
:1037E000A71B0F931F9341E050E060E070E08A0157
:1037F0009B0104C0000F111F221F331F8A95D2F7AF
:10380000C901B8011F910F910C94A71B0F931F932F
:1038100041E050E060E070E004C0440F551F661FB7
:10382000771F8A95D2F78091AB019091AC01A0915E
:10383000AD01B091AE018A019B01082B192B2A2BF7
:103840003B2BC901B8011F910F910C94A71B0F933B
:103850001F9341E050E060E070E004C0440F551F4A
:10386000661F771F8A95D2F74095509560957095A1
:103870008091AB019091AC01A091AD01B091AE01EE
:103880008A019B01082319232A233B23C901B8017C
:103890001F910F910C94A71B0F931F9341E050E0D1
:1038A00060E070E004C0440F551F661F771F8A95C3
:1038B000D2F78091AB019091AC01A091AD01B09194
:1038C000AE018A019B01082719272A273B27C90136
:1038D000B8011F910F910C94A71B0F931F93009198
:1038E000AB011091AC012091AD013091AE01602B84
:1038F000712B822B932B1F910F910C94A71B0F936D
:103900001F930091AB011091AC012091AD0130915A
:10391000AE0160237123822393231F910F910C9496
:10392000A71B0F931F930091AB011091AC01209145
:10393000AD013091AE0160277127822793271F9137
:103940000F910C94A71B0895CF92DF92EF92FF92F4
:103950000F931F93CF93DF938C01C090AF01D09052
:10396000B001E090B101F090B2014091AB015091F3
:10397000AC016091AD017091AE01C42AD52AE62A4E
:10398000F72ACFE1D0E0D701C6010C2E04C0B695CE
:10399000A795979587950A94D2F780FF07C0B8013D
:1039A0008C2F0E94BC1E8130910531F4219758F76D
:1039B000B80180E00E94BC1EDF91CF911F910F9152
:1039C000FF90EF90DF90CF90089520910D013091FE
:1039D0000E01F90132969FEF40E05191581789F09E
:1039E0009F3F19F4511101C0942F4F5F4630A9F742
:1039F0009F3F39F0F901E90FF11D97FDFA95828398
:103A00000895089520910D0130910E01F90132962B
:103A1000285F3F4F9081981301C010823196E217C2
:103A2000F307C1F7089581E090E0E0910D01F09176
:103A30000E01E80FF91F1082019688309105A9F751
:103A400008958091BD0108959091BD01892B8093C7
:103A5000BD01089580959091BD0189238093BD019A
:103A600008958093BD0108951092BD01089590912D
:103A7000BC01892B8093BC01089580959091BC0175
:103A800089238093BC0108951092BC01089580930E
:103A9000B30108951092B301089580910D019091A2
:103AA0000E01FC0131969C01285F3F4F80E091910F
:103AB00091118F5FE217F307D1F70895E0910D019F
:103AC000F0910E018091BD018083E0910D01F09194
:103AD0000E0190818091BC01892B80838091B3017C
:103AE000882361F0E0910D01F0910E019081892B06
:103AF00080830E944D1D81111092B30180910D01B0
:103B000090910E010C94A311909335018093340190
:103B100008958295982F9C7C292F26952695982F7D
:103B20009373990F990F922B892F8A7A86959575A1
:103B3000990F892B08950895CF93DF9300D000D07B
:103B40001F92CDB7DEB70F900F900F900F900F9090
:103B5000DF91CF910895089508950C94EB12809110
:103B6000D301843021F11092BF0120E488E190E07C
:103B70000FB6F894A895809360000FBE2093600064
:103B800083B7817F846083BF83B7816083BF78946C
:103B9000889583B78E7F83BF0FB6F894A8958091E0
:103BA0006000886180936000109260000FBE0895ED
:103BB00008950895CF930E94D81D0E94F2070E9495
:103BC000D91DC0E08C2F0E94F008811104C0CF5F86
:103BD000C031C1F701C081E0CF9108950C94AD17B9
:103BE0001F920F920FB60F9211248F939F93AF9352
:103BF000BF938091BF01811113C08091C00190914A
:103C0000C101A091C201B091C3014196A11DB11D96
:103C10008093C0019093C101A093C201B093C301EE
:103C2000BF91AF919F918F910F900FBE0F901F90FA
:103C3000189582E084BD93E095BD9AEF97BD80937F
:103C40006E0008952FB7F8948091C0019091C10142
:103C5000A091C201B091C3012FBF08952FB7F8946E
:103C60006091C0017091C1018091C2019091C30126
:103C70002FBF0895CF92DF92EF92FF920F931F9381
:103C80002FB7F8944091C0015091C1016091C201D9
:103C90007091C3012FBF6A017B01EE24FF248C01C8
:103CA00020E030E0C016D106E206F30610F44150E1
:103CB00051099A01281B390BC9011F910F91FF90DF
:103CC000EF90DF90CF9008951F920F920FB60F9252
:103CD00011248F939F93AF93BF938091C0019091D4
:103CE000C101A091C201B091C3010196A11DB11DF6
:103CF0008093C0019093C101A093C201B093C3010E
:103D0000BF91AF919F918F910F900FBE0F901F9019
:103D100018950E94EB0EF8942FEF87EA91E6215058
:103D200080409040E1F700C0000087E090EBDC01AC
:103D30008093DC019093DD01A093DE01B093DF015D
:103D40009CE088E10FB6F894A895809360000FBEC0
:103D500090936000FFCFE92FF0E093E0EE0FFF1F9C
:103D60009A95E1F7E80FF11DE855FF4F9491892FDF
:103D70008F7092959F700895CF93C82FCB010E94AA
:103D8000AB1E492F90E0242F30E054E0220F331F68
:103D90005A95E1F7282B392B2038310519F480E0AA
:103DA00090E017C0EC2FF0E023E0EE0FFF1F2A9504
:103DB000E1F74770E40FF11D34E0EE0FFF1F3A9575
:103DC000E1F7E80FF91FEE0FFF1FE050F84985916A
:103DD0009491CF91089580E090E0089508958091A6
:103DE000C60180FF0CC08091120190E065E070E098
:103DF0000E94A72695958795959587952EC081FF5A
:103E00000AC08091120190E065E070E00E94A72650
:103E10009595879522C082FF08C08091120190E09D
:103E200065E070E00E94A72618C02091C7012223F8
:103E3000D1F030911101231780F78091120190E0A9
:103E400065E070E00E94A726622F70E00E94A7261E
:103E5000632F70E00E94C426CB018038910530F4B6
:103E6000009731F0089585E090E008958FE7089578
:103E700081E008958091C60180FF08C06091100123
:103E800070E0759567957595679523C081FF06C0AD
:103E90006091100170E0759567951BC082FF04C0AA
:103EA0006091100170E012C06091C7016623D1F0EB
:103EB00020910F016217A0F78091100170E090E04F
:103EC0000E94A726622F70E00E94C4266038710508
:103ED00028F46115710521F0862F08958FE7089564
:103EE00081E0089561E070E0F4CF803F21F40E940A
:103EF000EF1E819504C0813F29F40E94EF1E80933C
:103F0000CA010895823F21F40E94EF1E819504C0EA
:103F1000833F29F40E94EF1E8093C9010895893FD1
:103F200019F40E943A1F05C08A3F31F40E943A1FDB
:103F300081958093CB0108958B3F21F40E943A1F15
:103F4000819504C08C3F29F40E943A1F8093CC01D4
:103F50000895843F21F48091C801816017C0853F96
:103F600021F48091C801826011C0863F21F48091C4
:103F7000C80184600BC0873F21F48091C80188602C
:103F800005C0883F31F48091C80180618093C801E9
:103F900008958D3F21F48091C60181600BC08E3F52
:103FA00021F48091C601826005C08F3F29F4809181
:103FB000C60184608093C6010895803F39F48091E2
:103FC000CA0187FF6CC01092CA0169C0813F29F401
:103FD0008091CA011816BCF362C09091C901823F5A
:103FE00029F497FF5CC01092C90159C0833F19F4AE
:103FF0001916CCF354C0893F41F48091CB011816B7
:104000000CF04DC01092CB014AC08A3F29F4809138
:10401000CB0187FF44C0F6CF8B3F39F48091CC01B0
:1040200087FF3DC01092CC013AC08C3F29F48091AB
:10403000CC011816BCF333C0843F21F48091C80131
:104040008E7F17C0853F21F48091C8018D7F11C0FC
:10405000863F21F48091C8018B7F0BC0873F21F4FC
:104060008091C801877F05C0883F31F48091C801E5
:104070008F7E8093C80113C08D3F21F48091C601CB
:104080008E7F0BC08E3F21F48091C6018D7F05C0CD
:104090008F3F29F48091C6018B7F8093C601809168
:1040A000C90181110EC08091CA0181110AC080919D
:1040B000CB01811106C08091CC01811102C0109208
:1040C000C70108958091BE0183FF7EC08BE894E014
:1040D0000E948D058091C8011F928F9386E894E01D
:1040E0009F938F930E94260684E894E00E948D059A
:1040F0008091C901282F082E000C330B3F938F931A
:1041000081E894E09F938F930E9426068FE794E0C6
:104110000E948D058091CA01282F082E000C330BB8
:104120003F938F938CE794E09F938F930E94260692
:104130008AE794E00E948D058091CB01282F082EFC
:10414000000C330B3F938F9387E794E09F938F93FB
:104150000E94260685E794E00E948D058091CC019F
:10416000282F082E000C330B3F938F9382E794E0A7
:104170009F938F930E9426068FE694E00E948D0500
:104180008091C7011F928F938CE694E09F938F9349
:104190000E9426068AE694E00E948D058091C60161
:1041A0001F928F9387E694E09F938F930E94260639
:1041B00084E694E00E948D058DB79EB74C960FB6AD
:1041C000F8949EBF0FBE8DBF88EC91E00E94EC1169
:1041D0000E94221E9093C5018093C40108951F93ED
:1041E000CF93DF938091C4019091C5010E943A1E44
:1041F000FC012091C701222329F090911301892FFE
:1042000090E007C08091140190E06AE070E00E94A5
:10421000A726E817F90708F485C08091C901C09165
:10422000CA01D091CB011091CC01811107C0C111FD
:1042300075C0D11173C0111171C074C02F3F19F036
:104240002F5F2093C701181624F40E94EF1E80935D
:10425000C9018091C90187FF05C00E94EF1E8195A9
:104260008093C9011C1624F40E94EF1E8093CA019A
:104270008091CA0187FF05C00E94EF1E819580933F
:10428000CA016091C901662331F1C091CA01CC23F2
:1042900011F1062E000C770B880B990B0E94A625B6
:1042A00023E333E343E35FE30E940A260E946E2583
:1042B0006093C9016C2FCC0F770B880B990B0E9470
:1042C000A62523E333E343E35FE30E940A260E942B
:1042D0006E256093CA011D1624F40E943A1F809334
:1042E000CB018091CB0187FF05C00E943A1F8195C9
:1042F0008093CB01111624F40E943A1F8093CC01C5
:104300008091CC0187FF05C00E943A1F8195809360
:10431000CC01DF91CF911F910C9462202F3F09F0C7
:104320008FCF97CFDF91CF911F910895E8ECF1E007
:1043300085E0DF011D928A95E9F71092C70110927E
:10434000C60108958EEA96E00E948D051F9281E0D5
:104350008F931F9285E08F9380E696E09F938F93D3
:104360000E9426060F900F900F900F900F900F90C5
:1043700008958330E9F128F4813061F0823009F149
:104380000895853009F462C008F449C0863009F404
:1043900074C0089580911401262F30E0280F311D3C
:1043A0002F3F310524F4680F6093140103C08FEF91
:1043B00080931401809114011F928F9389E995E0F5
:1043C00072C080911301262F30E0280F311D2F3F3E
:1043D000310524F4680F6093130103C08FEF8093BD
:1043E0001301809113011F928F9387E895E05BC0C2
:1043F00080911201262F30E0280F311D2F3F31050B
:1044000024F4680F6093120103C08FEF80931201B0
:10441000809112011F928F9384E795E044C08091B0
:104420001101262F30E0280F311D2F3F310524F4D4
:10443000680F6093110103C08FEF80931101809189
:1044400011011F928F938FE595E02DC0809110018F
:10445000262F30E0280F311D2F3F310524F4680F3F
:104460006093100103C08FEF8093100180911001C1
:104470001F928F9386E495E016C080910F01262F3E
:1044800030E0280F311D2F3F310524F4680F609371
:104490000F0103C08FEF80930F0180910F011F92D6
:1044A0008F938BE295E09F938F930E9426060F9047
:1044B0000F900F900F900895833081F128F4813090
:1044C00059F08230D1F00895853009F449C0B8F12F
:1044D000863009F456C0089580911401681720F4BD
:1044E000861B8093140102C0109214018091140164
:1044F0001F928F938CE195E054C08091130168174F
:1045000020F4861B8093130102C010921301809146
:1045100013011F928F938AE095E043C080911201AE
:10452000681720F4861B8093120102C010921201BA
:10453000809112011F928F9387EF94E032C0809197
:104540001101681720F4861B8093110102C010929C
:104550001101809111011F928F9382EE94E021C08E
:1045600080911001681720F4861B8093100102C00F
:1045700010921001809110011F928F9389EC94E0AA
:1045800010C080910F01681720F4861B80930F01E3
:1045900002C010920F0180910F011F928F938EEA3B
:1045A00094E09F938F930E9426060F900F900F9098
:1045B0000F900895CF93C82F1F928F9383EB97E0AE
:1045C0009F938F930E94260681E090E0A0E0B0E0E8
:1045D000BC01CD0104C0660F771F881F991FCA95C3
:1045E000D2F70E94B41B0F900F900F900F90CF91B5
:1045F0000C94AD17CF93873288F58E3108F00BC13C
:104600008E3009F487C0D8F4873009F460C08B304D
:1046100009F44FC0863009F002C18091BE01817F4C
:104620008E7F8093BE0188EB97E00E948D058CE61B
:104630009AE00E948D0581E08093CE0146C08631CC
:1046400009F4B0C020F4803109F47AC0E8C089319F
:1046500009F491C08B3109F449C0E1C0883349F1B4
:1046600050F4893209F4D5C0853309F4D2C08732B9
:1046700009F0D5C0CEC0833409F4CBC028F48A3306
:1046800008F4CDC08953C8C0883409F0C8C00E945E
:10469000AD178BE59AE00E948D052FEF83ED90E337
:1046A000215080409040E1F700C000000E94891E28
:1046B0000CC08FED97E041C082E49AE00E948D0526
:1046C0008091BE0181608093BE01C1E0ADC0809148
:1046D000BE01C82FC17080FFEFCF8EE49AE00E9428
:1046E0008D058091BE01817F8E7F3FC09091BE017C
:1046F00091FBCC27C0F981E0C827892FC0FB81F945
:104700008093BE01CC2319F085E39AE029C087E2AB
:104710009AE013C09091BE0192FBCC27C0F981E0D2
:10472000C827892FC0FB82F98093BE01CC2319F0E2
:1047300088E19AE015C088E09AE00E948D05C5CF17
:104740009091BE0193FBCC27C0F981E0C827892F47
:10475000C0FB83F98093BE01CC2351F08CEF99E02C
:104760000E948D058091BE0181608093BE015CC076
:104770008FEE99E0E2CF80EE99E00E948D058DEBFF
:1047800099E00E948D0588E799E00E948D0581E5FA
:1047900099E00E948D058CE099E00E948D058DEDD9
:1047A00098E0CBCF8FEC98E00E948D050E94971186
:1047B0001F928F9385EB98E09F938F930E9426061C
:1047C00080910C011F928F938EE998E09F938F93B5
:1047D0000E94260680915B011F928F938BE898E0E0
:1047E0009F938F930E9426060E942E1E9F938F9365
:1047F0007F936F9384E798E09F938F930E942606A0
:104800008DB79EB742960FB6F8949EBF0FBE8DBF70
:104810005CCF80E001C08D510E94DA2256CF82E742
:1048200098E00E948D05C0E08C2FCF91089580E024
:10483000089580E00895CF93C82F8091CE018130F4
:1048400069F020F0823009F449C040C167E08FE090
:104850000E94DB08882309F43FC106C067E08FE0AF
:104860000E94DB08882361F08C2F0E94172481119D
:1048700004C08C2F0E94FA222FC081E090E02CC04F
:104880008C2F0E941924811126C0C431E1F070F4EC
:10489000CB3081F0C031D1F40E94A2218BEA97E0A5
:1048A0000E948D0582E08093CE0115C0C93259F077
:1048B000C83361F488EB97E00E948D058FEA97E09A
:1048C0000E948D0508C01092CE0104C189EA97E0CC
:1048D0000E948D05FFC081E08170FEC0C43228F5C2
:1048E000CE3108F0C1C0CB30A1F1D0F4C73009F00F
:1048F000D3C08EE18093140182E3809313018AE098
:104900008093120184E18093110188E0809310016B
:1049100088E280930F018FE496E00E948D05BFC06E
:10492000C33149F1C431C1F0B7C0CB3409F4A9C0D7
:1049300028F4C93289F0C83361F0AEC0C13509F43A
:104940009EC0C23509F499C0CE3409F0A5C06AE012
:104950009EC00E94A221A3C08091CD01882319F09E
:104960001092CD019CC08CE596E00E948D0581E0FF
:104970008093CE01B1C086E396E00E948D0584E26B
:1049800096E00E948D05809114011F928F9381E221
:1049900096E09F938F930E9426068FE196E00E94F7
:1049A0008D058DE096E00E948D05809113011F9288
:1049B0008F938AE096E09F938F930E94260688E06B
:1049C00096E00E948D0589EF95E00E948D0580910B
:1049D00012011F928F9386EF95E09F938F930E9411
:1049E000260684EF95E00E948D0583EE95E00E94F7
:1049F0008D05809111011F928F9380EE95E09F931A
:104A00008F930E9426068EED95E00E948D0589EC1D
:104A100095E00E948D05809110011F928F9386EC86
:104A200095E09F938F930E94260684EC95E00E9468
:104A30008D058DEA95E00E948D0580910F011F92F2
:104A40008F938AEA95E09F938F930E94260688EAC7
:104A500095E00E948D058DB79EB748960FB6F894E5
:104A60009EBF0FBE8DBF1BC0CE51EC2FF0E0E75DA7
:104A7000FE4F80818093CD0112C061E003C061E0F0
:104A800006C06AE08091CD010E94B92108C08091E2
:104A9000CD010E945C2203C08DE496E013C080919A
:104AA000CD01882369F01F928F9387E496E09F934E
:104AB0008F930E9426060F900F900F900F9004C0C6
:104AC00084E496E00E948D0581E006C01092CE013C
:104AD00080E002C080E000CFCF9108950E9475254C
:104AE0006894B1110C94042608950E94E92588F079
:104AF0009F5798F0B92F9927B751B0F0E1F0660FA2
:104B0000771F881F991F1AF0BA95C9F714C0B130E2
:104B100091F00E940326B1E008950C940326672FBC
:104B2000782F8827B85F39F0B93FCCF38695779511
:104B30006795B395D9F73EF49095809570956195FA
:104B40007F4F8F4F9F4F0895E89409C097FB3EF425
:104B500090958095709561957F4F8F4F9F4F9923CA
:104B6000A9F0F92F96E9BB279395F6958795779548
:104B70006795B795F111F8CFFAF4BB0F11F460FF08
:104B80001BC06F5F7F4F8F4F9F4F16C0882311F060
:104B900096E911C0772321F09EE8872F762F05C074
:104BA000662371F096E8862F70E060E02AF09A950F
:104BB000660F771F881FDAF7880F9695879597F904
:104BC000089557FD9058440F551F59F05F3F71F0FD
:104BD0004795880F97FB991F61F09F3F79F0879564
:104BE0000895121613061406551FF2CF4695F1DFED
:104BF00008C0161617061806991FF1CF869571057D
:104C0000610508940895E894BB2766277727CB01B0
:104C100097F908950E941C260C9496260E948826D7
:104C200038F00E948F2620F0952311F00C947F26F7
:104C30000C9485260C9404260E94E12578F3992390
:104C4000C9F35523B9F3950F50E0551FAA27EE2756
:104C5000FF27BB2700240894679520F4E20FF31F79
:104C6000B41F0A1E220F331F441FAA1F6695A9F7FF
:104C7000779530F4F30FB41F0A1E121E08F46395E3
:104C8000330F441FAA1F221F769599F7879520F4AA
:104C9000B40F0A1E121E631F440FAA1F221F331FC8
:104CA0008695A9F7862F712D602D11249F575040AE
:104CB0009AF0F1F088234AF0EE0FFF1FBB1F661F2A
:104CC000771F881F91505040A9F79E3F510580F0F3
:104CD0000C947F260C9404265F3FE4F3983ED4F3B3
:104CE000869577956795B795F795E7959F5FC1F797
:104CF000FE2B880F911D9695879597F9089597F942
:104D00009F6780E870E060E008959FEF80EC089571
:104D100000240A941616170618060906089500249A
:104D20000A9412161306140605060895092E039414
:104D3000000C11F4882352F0BB0F40F4BF2B11F488
:104D400060FF04C06F5F7F4F8F4F9F4F0895002417
:104D5000552704C0080E591F880F991F009729F086
:104D600076956795B8F37105B9F7802D952F08955D
:104D7000991B79E004C0991F961708F0961B881FAD
:104D80007A95C9F78095089597FB072E16F400943D
:104D900007D077FD09D00E94DE2607FC05D03EF43F
:104DA000909581959F4F0895709561957F4F0895D7
:104DB000EE0FFF1F0590F491E02D0994AA1BBB1B79
:104DC00051E107C0AA1FBB1FA617B70710F0A61B0B
:104DD000B70B881F991F5A95A9F780959095BC012C
:084DE000CD010895F894FFCF06
:104DE800FFFF5C0A4D0B2A0BF60AC20A01B4012820
:104DF80008140A321E404D3622FF03B2037C035AC0
:104E080003E602FF02180331030102030405060743
:044E18000809000085
:106800000000EA44E944E2440400050006000700F1
:10681000080009000A000B000C000D000E000F001C
:1068200010001100120013001400150016001700CC
:10683000180019001A001B001C001D001E001F007C
:10684000200021002200230024002500260027002C
:10685000280029002A002B002C002D002E002F00DC
:10686000300031A132003300340035A1360037004A
:10687000380082003A003B003C003D003E003F00F3
:1068800040004100420043004400450046004700EC
:10689000480049004A004B004C004D004E004F009C
:1068A000500051005200530067005400550056003C
:1068B000580059005A005B005C005D005E005F00FC
:1068C0006000610062006300640000005700000087
:1068D000CD440000000000000000000000000000A7
:1068E0000000000000007300000000000000000035
:1068F000E000E100E200E300E400E500E600E7007C
:106900000100010001000100EA4401000100E2442D
:106910000100010001000100460001004A004B0097
:10692000010001004700480001000100E9440100A6
:106930000100010001000100010001003A003B00DC
:106940003C003D003E003F0040004100420043004B
:10695000010001004C00010001004400450052000C
:1069600049000100010050004F0001004D004E00A1
:1069700051000100010001000100010001000100BF
:1069800001000100010001000100010001000100FF
:1069900001000100010001000100010001004D00A3
:1069A0004A004E004B0001000100010001000100FF
:1069B00001000100010001000100010001000100CF
:1069C00001000100010001000100010001000100BF
:1069D00001000100010001000100010001000100AF
:1069E000010001000100010001000100010001009F
:1069F000010001000100010001000100010001008F
:00000001FF
